:020000040800F2
:100000006022002005010008992E0008492C0008F4
:10001000952E000857070008F76000080000000050
:10002000000000000000000000000000B9330008DC
:1000300035080008000000008F330008BB330008BB
:100040001F0100081F0100081F0100081F01000810
:100050001F0100081F0100081F0100081F01000800
:100060001F0100081F0100081F0100081F010008F0
:100070001F0100081F0100081F0100081F010008E0
:100080001F0100081F0100081F0100081F010008D0
:10009000416000081F0100081F0100081F0100083F
:1000A0001F0100081F0100081F0100081F010008B0
:1000B0001F0100081F0100081F0100081F010008A0
:1000C0001F0100081F0100081F0100081F01000890
:1000D0001F010008093A00081F0100081F0100085D
:1000E0001F0100081F0100081F010008DFF810D0E1
:1000F00000F042F900480047FD630008AFF30080BC
:10010000602200200648804706480047FEE7FEE7D9
:10011000FEE7FEE7FEE7FEE7FEE7FEE7FEE7FEE7B7
:100120004F340008ED00000840EA01039B0703D0AC
:1001300009E008C9121F08C0042AFAD203E011F826
:10014000013B00F8013B521EF9D27047D2B201E0E8
:1001500000F8012B491EFBD270470022F6E710B5CC
:1001600013460A4604461946FFF7F0FF204610BD25
:100170000FB400B58DB010A909900B9000914FF00D
:10018000FF300A9000200C90054806900548079023
:100190006A4609A80F9900F0C1F80DB05DF814FB8C
:1001A00039030008570300082DE9FF5F1D464FF093
:1001B000FF3BD5E9014691465F464FF00008A9692B
:1001C0007F1C01988847296A824688470028F6D113
:1001D000BAF1FF3F0CD024F4C064002E19DD600694
:1001E00014D5BAF12B0F09D0BAF12D0F0ED103E0BF
:1001F000584604B0BDE8F09F44F48064A9697F1CB0
:1002000001988847761E8246002E02DDBAF1300F33
:1002100003D0B9F1000F26D032E0A969761E44F46C
:1002200000747F1C019888478246002E05DDBAF1D4
:10023000780F06D0BAF1580F03D0B9F1000F10D0E3
:100240001EE0B9F1000F02D0B9F1100F18D1A96961
:10025000761E24F400747F1C019888478246102083
:1002600002E0082000E00A20814609E008FB0908B6
:10027000A969761E44F400747F1C01988847824661
:10028000002E05DD4946504600F034F80028EDDA2E
:10029000E96901988847A00502D46FF00100A8E73A
:1002A000E00725D1600613D5600502D5C8F100002E
:1002B00000E0404629680A1D2A600968220501D528
:1002C000087015E0220701D5088011E008600FE0F2
:1002D0002868011D29600068210502D580F800808A
:1002E00006E0210702D5A0F8008001E0C0F80080F8
:1002F00038467EE73A2800D2303820F02002412AE2
:1003000001D3A2F13700884201D34FF0FF3070478C
:10031000026811441378016018467047D16004499F
:1003200051610449116200211161114600F03CB88D
:10033000110300089D030008426842B1016811F8EA
:10034000013B23B1521EC0E900121846704701213B
:10035000C160881E704742685AB1C368016843B9DA
:1003600083688B4205D0491E521CC0E90012002050
:1003700070474FF0FF307047064C074D06E0E068CD
:1003800040F0010394E8070098471034AC42F6D3DC
:10039000FFF7B0FE906A0008B06A0008C0B24FF4E0
:1003A000F05100F099B900002DE9F34F8BB04FF0F8
:1003B000000801F10C000C464FF0010B46460DF110
:1003C000080A01906269012101989047051E2DD00D
:1003D000252D2CD0216A8847C0B16269012101987E
:1003E0009047216A88470028F7D1411E6269019829
:1003F000904700E0761CA1690B988847216A8847DE
:100400000028F7D1E1690B988847DBE7A1690B98D1
:1004100088470746A84201D1761CD3E7E1690B98CB
:1004200088477F1C02D1B8F1000F6FD047E1002749
:1004300062693D463946019890472A2804D162698D
:100440000121019890470125DFF888926269012116
:1004500001989047A0F130010A290AD24F45E5DC06
:1004600007EB870100EB4107303FDFD445F0100573
:10047000ECE7E90601D46FF000476C280AD04C285D
:1004800014D0682815D06A280DD074281CD07A287A
:100490001AD01DE062690121019890476C2802D0B2
:1004A00045F0040514E045F002050DE045F0200597
:1004B0000AE06269012101989047682802D045F05E
:1004C000080505E045F4006562690121019890473F
:1004D000C4E9015765283DD019DC58287AD00CDCD6
:1004E000452837D004DC252826D0412831D131E0F9
:1004F00046282FD047282CD12CE05B2877D06128C4
:1005000028D063287CD0642823D15AE0D1E06F281A
:1005100048D008DC66281DD067281BD0692821D068
:100520006E2816D127E0702845D0732868D075282A
:1005300047D078280DD14DE0A1690B988847054632
:1005400025283FF469AFE1690B9888476D1C3FF49B
:100550006AAFB4E023466A466FF001000B99AFF32F
:1005600000809FE045F040006060A80723464FF000
:10057000000236D43EE0E8077FF447AF2068011D53
:1005800021600068290501D506701BE7290701D500
:10059000068017E7A90703D5F117C0E9006111E745
:1005A00006600FE745F040006060A80723464FF063
:1005B000080216D41EE040F60E0125EA0100606034
:1005C00016E045F040006060A80723464FF00A029D
:1005D00007D40FE045F040006060A80708D5234627
:1005E00010226FF001000B99AFF300805AE007E092
:1005F000234610226FF001000B99FFF7D5FD51E063
:100600004FF000094F464B46632802D05B2807D0C5
:1006100041E02079C00601D40120A06001273AE022
:1006200062690121019890475E2805D14FF00109C8
:100630006269494601989047216939B900210A4603
:10064000534643F82120491C0829FADBB0B321693D
:1006500069B9C11700EBD16253110AEB830122F093
:100660001F02821A01200B68904003430B606269ED
:100670000121019890475D28E8D1B9F1000F09D018
:100680000020514651F82020D24341F82020401C40
:100690000828F7DB02AB224600976FF001000B99A8
:1006A000AFF3008000280CDA401C08D1BBF1000F2A
:1006B00005D04FF0FF300DB0BDE8F08FFFE74046AA
:1006C000F9E7E90701D108F1010806444FF0000BF2
:1006D00078E60000CCCCCC0C7F2801D9002208E0C1
:1006E000064A02EB5002C007127800D1120902F04C
:1006F0000F02012090400840704700004F6A000838
:1007000070B58C1810F8015B15F0070301D110F8D3
:10071000013B2A1106D110F8012B03E010F8016B00
:1007200001F8016B5B1EF9D12B0705D40023521E83
:100730000DD401F8013BFAE710F8013BCB1A921CEB
:1007400003E013F8015B01F8015B521EF9D5A142E9
:10075000D8D3002070BD00BFFEE70346042B15D0A0
:1007600007DC7BB1012B0ED0022B0DD0032B12D155
:100770000BE0202B0BD0212B0AD0222B09D0232BCE
:1007800009D107E008E007E006E005E004E003E047
:1007900002E001E000E000BF00BF00207047002041
:1007A0007047000010B500220449054803F073FAB1
:1007B0000449034803F068FA002010BD400B0020F4
:1007C0007C0200204007002070B505460C46154904
:1007D000098820680844B0F5007F14D81249114BED
:1007E0001B88C81829462268FFF79EFC20880D49FF
:1007F000098808440B4908802068402808D2012055
:100800000A49087004E0002006490880074908707A
:100810002946074803F038FA054803F011FA00208A
:1008200070BD000058000020400F00205A0000203A
:100830007C020020704772B600BFFEE770B50A4820
:100840000468001D0568001D0668344454B1082280
:100850000649204602F0FAF90422044910312846DC
:1008600002F0F4F970BD0000E8F7FF1F3E00002021
:100870000146002291F82100022808D00420886354
:1008800000BF002081F8200000BF012070470868E9
:10089000006820F00E000B6818600868006820F0FF
:1008A00001000B68186091F8403001209840CB6B34
:1008B0005860012081F8210000BF002081F820004D
:1008C00000BF1046E2E7000070B50446002594F82A
:1008D0002100022803D00420A063012548E02068FD
:1008E000006820F00E00216808602068006820F091
:1008F0000100216808601F492068884201D1012059
:1009000026E01C4914312068884201D110201FE0E4
:10091000184928312068884201D1801518E015490E
:100920003C312068884201D1801411E011495031D6
:100930002068884202D14FF4803009E00D496431CB
:100940002068884202D14FF4801001E04FF080709F
:10095000084908394860012084F8210000BF0020C0
:1009600084F8200000BF606B10B12046616B88479F
:10097000284670BD0800024070B5044600F0AEF98C
:1009800006462546681C10B104480078054400BF9F
:1009900000F0A4F9801BA842FAD370BD74000020B7
:1009A0002DE9F8470346002294466EE14FF0010816
:1009B00008FA02F4D1F8008008EA0400A0427DD1D0
:1009C000DFF8DCA2D1F80480A8EB0A09D0453AD0C0
:1009D00014DCB8F1030F50D009DCB8F1000F31D0AE
:1009E000B8F1010F1CD0B8F1020F49D120E0B8F1E5
:1009F000110F18D0B8F1120F42D11EE0B9F5881FBF
:100A000025D006DCB9F5803F20D0B9F5801F37D15D
:100A10001AE0B9F5001F18D0B9F5041F30D117E05E
:100A2000D1F80CC02DE0D1F80C8008F1040C28E0BE
:100A3000D1F80C8008F1080C23E0D1F80C8008F103
:100A40000C0C1EE000BF00BF00BF00BF00BF00BF16
:100A5000D1F80880B8F1000F02D14FF0040C0BE080
:100A6000D1F80880B8F1010F03D14FF0080C1C61D8
:100A700002E04FF0080C5C6103E04FF0000C00E076
:100A800000BF00BFFF2801D8984601E003F1040829
:100A90004646FF2802D84FEA820803E0A2F1080880
:100AA0004FEA88084746D6F800804FF00F0909FA48
:100AB00007F928EA09080CFA07F900E088E048EA93
:100AC0000908C6F80080D1F8048008F08058B8F111
:100AD000805F7DD100BFDFF8CC81D8F8188048F066
:100AE0000108DFF8C091C9F81880C846D8F8188006
:100AF00008F00108CDF8008000BF00BF4FEAB93808
:100B00004FEA920958F829504FEA82784FEA18794B
:100B10004FF00F0808FA09F825EA0805DFF8888180
:100B2000434502D14FF0000816E0DFF880814345CD
:100B300002D14FF001080FE0DFF87481434502D184
:100B40004FF0020808E0DFF86C81434502D14FF016
:100B5000030801E04FF004084FEA82794FEA19795F
:100B600008FA09F848EA0505DFF84C814FEA9209CE
:100B700048F82950D1F8048008F48018B8F5801F8F
:100B80000AD1DFF83881D8F8008048EA0008DFF899
:100B90002C91C9F8008009E0DFF82081D8F80080A6
:100BA00028EA0008DFF81491C9F80080D1F8048021
:100BB00008F40018B8F5001F10D1DFF8008108F123
:100BC0000408D8F8008048EA0008DFF8F09000E058
:100BD0005AE009F10409C9F800800DE0DFF8DC8073
:100BE00008F10408D8F8008028EA0008DFF8CC9063
:100BF00009F10409C9F80080D1F8048008F400382C
:100C0000B8F5003F0ED1DFF8B480A8F10408D8F899
:100C1000008048EA0008DFF8A490A9F10409C9F8A7
:100C200000800DE0DFF89480A8F10408D8F8008077
:100C300028EA0008DFF88490A9F10409C9F80080C7
:100C4000D1F8048008F48038B8F5803F0ED1DFF881
:100C50006C80A8F10808D8F8008048EA0008DFF89E
:100C60005C90A9F10809C9F800800DE0DFF84C801C
:100C7000A8F10808D8F8008028EA0008DFF83C90BE
:100C8000A9F10809C9F80080521CD1F8008028FA9F
:100C900002F8B8F1000F7FF489AEBDE8F8870000D4
:100CA000000011100010024000080140000C01403B
:100CB00000100140001401400800014008040140F8
:100CC000024693680B400BB1012000E00020704702
:100CD0000AB1016101E00B0403617047014800683B
:100CE000704700006C000020034800680349097841
:100CF00008440149086070476C000020740000201F
:100D000010B50848006840F010000649086003204C
:100D100000F0A8F80F2000F007F800F02BF80020F2
:100D200010BD00000020024070B504460E48007857
:100D30004FF47A71B1FBF0F00C490968B1FBF0F5A2
:100D4000284601F0ABFB08B1012070BD102C07D282
:100D500000222146501E00F047F80548046001E0DB
:100D60000120F2E70020F0E7740000207800002066
:100D70007000002008B500BF1148806940F00100F4
:100D80000F4988610846806900F00100009000BFAB
:100D900000BF00BF0846C06940F08050C8610846E7
:100DA000C06900F08050009000BF00BF00BF05493F
:100DB000486820F0E06040F00070486000BF08BD67
:100DC000001002400000014001460846002809DBEF
:100DD00000F01F0301229A4043099B0003F1E02326
:100DE000C3F8002100BF70472DE9F05F80460D4633
:100DF0001646002705F082F9074639462A4633464B
:100E000001F00700C0F1070ABAF1040F02D94FF050
:100E1000040A01E0C0F1070AD14600F1040ABAF160
:100E2000070F02D24FF0000A01E0A0F1030AD446F6
:100E30004FF0010A0AFA09FAAAF1010A0AEA020ABB
:100E40000AFA0CFA4FF0010B0BFA0CFBABF1010B99
:100E50000BEA030B4AEA0B042146404605F056F91B
:100E6000BDE8F09F00BF00F00702064B19684FF67F
:100E7000FF031940044B0B4343EA0221014B196065
:100E800000BF70470CED00E00000FA0570B50546A4
:100E90000C4604F08000802808D104F0070000EB25
:100EA000800605F1280000EBC60105E004EB84068E
:100EB00005F5B47000EBC6011AB900200873CB80A9
:100EC00004E0012008730B81180C4881002070BDDC
:100ED000704770B504460D4605EB850304F1280103
:100EE00001EBC3014A692946D4F8EC0203F046FA43
:100EF00070BD70B504460D4605EB850304F5B4716D
:100F000001EBC3014A692946D4F8EC0203F0B6FAB2
:100F100070BD70B504460E4606F0800080280AD1E8
:100F200006F0070000EB800104F1280000EBC1058A
:100F30000120687009E006F0070000EB800104F56D
:100F4000B47000EBC1050020687006F0070028703F
:100F500000BF94F8A802012801D1022070BD012031
:100F600084F8A80200BF2946206804F041F900BFB8
:100F7000002084F8A80200BF00BFEFE770B5044668
:100F80000E4606F00F006168884201D9012070BD4D
:100F900006F0800080280AD106F0070000EB8001EF
:100FA00004F1280000EBC1050120687009E006F09B
:100FB000070000EB800104F5B47000EBC1050020D0
:100FC00068700020A87006F00700287000BF94F831
:100FD000A802012801D10220D9E7012084F8A80243
:100FE00000BF2946206804F05FFA00BF002084F8A3
:100FF000A80200BF00BFCAE72DE9F04105460C4634
:10100000174607F48040002850D02868B0F85010E8
:10101000207801EBC000801C296801F5806131F85F
:101020001000C0F30906A069B04203D3A069801B79
:10103000A06101E00020A061A069A8B900BF2278EA
:101040005200296831F812104BF68F7201EA020043
:1010500080F4005040F4004141F0800123785B00AF
:101060002A6822F8131000BF07F04000A8B100BFA3
:1010700000BF22785200296831F8121048F68F72AA
:1010800001EA020040F4004141F0C00123785B0016
:101090002A6822F8131000BF00BF002E55D0228905
:1010A00061693346286804F0D7FF4EE02868B0F83D
:1010B0005010207801EBC000801D296801F5806187
:1010C00031F81000C0F30906A069B04203D3A0694B
:1010D000801BA06101E00020A061A069A8B900BF49
:1010E00022785200296831F812104BF68F7201EA0B
:1010F000020080F4005040F4004141F08001237868
:101100005B002A6822F8131000BF07F04000A8B95E
:1011100000BF00BF22785200296831F8121048F64B
:101120008F7201EA020040F4004141F0C0012378CF
:101130005B002A6822F8131000BF00BF2EB162893D
:1011400061693346286804F087FF3046BDE8F081C6
:101150002DE9F04705460C46904608F0400000286F
:101160007ED02868B0F85010207801EBC000801CB9
:10117000296801F5806131F81000C0F30907A06902
:10118000B84203D9A069C01BA06101E00020A061A2
:10119000A06900287ED100BF6078C0B900BF29686F
:1011A0002A68B2F8502011442278022303EBC202CD
:1011B00001F5806303EB420000BF0288C2F309021D
:1011C0000280028842F40042028000BF13E060788F
:1011D000012810D100BF28682A68B2F850201044B6
:1011E0002278022303EBC20200F5806303EB420185
:1011F00000220A8000BF00BF00BF29686078F8B9EC
:1012000000BF2B68D5F800C0BCF850C0634494F808
:1012100000C04FF0060909EBCC0C03F5806909EB1F
:101220004C0000BFB0F800C0CCF3090CA0F800C01F
:10123000B0F800C04CF4004CA0F800C000BF12E0B1
:10124000607801280FD12868B0F850000144207858
:10125000062303EBC00001F5806303EB400200E0CE
:10126000B7E00020108000BF21782846FFF731FE4C
:1012700008F48040002816D000BF00BF227852003A
:10128000296831F8121048F68F7201EA020040F422
:10129000004100E008E041F4814123785B002A68C6
:1012A00022F8131000BFD7E108F48040A8B100BFB6
:1012B00000BF22785200296831F8121048F68F7268
:1012C00001EA020040F4004141F4814123785B00CF
:1012D0002A6822F8131000BF00BF94F824000128E8
:1012E000E1D1606938446061E0693844E0612169B6
:1012F000206A884204D32669206A801B20620BE0A2
:10130000206A20B93E46002084F8240004E0002032
:1013100084F82400266A206200BF6078E8BB00BF22
:101320002A682968B1F850100A442178022303EB97
:10133000C10102F5806303EB4101084600BF038849
:10134000C3F3090303803E2E10D900BF710906F0D4
:101350001F0303B9491E03884FF4004C4CEA812C4B
:101360001FFA8CFC43EA0C03038014E026B90388BF
:1013700043F4004303800EE000BF710806F0010350
:1013800003B1491C03884FF6FF7C0CEA812C43EA29
:101390000C03038000BF00BF13E0FFE76078012863
:1013A0000FD100BF28682A68B2F850201044227874
:1013B000022303EBC20200F5806303EB42010E80BF
:1013C00000BF00BFB3B222896169286804F073FED0
:1013D00042E12868B0F85010207801EBC000801D71
:1013E000296801F5806131F81000C0F30907A06990
:1013F000B84203D3A069C01BA06101E00020A06136
:10140000A06900287ED100BF6078C0B900BF2968FC
:101410002A68B2F8502011442278022303EBC2025A
:1014200001F5806303EB420000BF0288C2F30902AA
:101430000280028842F40042028000BF13E060781C
:10144000012810D100BF28682A68B2F85020104443
:101450002278022303EBC20200F5806303EB420112
:1014600000220A8000BF00BF00BF29686078F8B979
:1014700000BF2B68D5F800C0BCF850C0634494F896
:1014800000C04FF0060909EBCC0C03F5806909EBAD
:101490004C0000BFB0F800C0CCF3090CA0F800C0AD
:1014A000B0F800C04CF4004CA0F800C000BF10E041
:1014B000607801280DD12868B0F8500001442078E8
:1014C000062303EBC00001F5806303EB400200201C
:1014D000108000BF21782846FFF7FBFC08F480400D
:1014E000002816D100BF00BF22785200296831F8C9
:1014F000121048F68F7201EA020040F4004141F4F4
:10150000814100E006E023785B002A6822F813108E
:1015100000BFA1E008F48040A8B900BF00BF227856
:101520005200296831F8121048F68F7201EA020061
:1015300040F4004141F4814123785B002A6822F89D
:10154000131000BF00BF94F8240001287ED1606909
:1015500038446061E0693844E0612169206A88426A
:1015600004D32669206A801B20620BE0206A20B920
:101570003E46002084F8240004E0266A0020206211
:1015800084F8240000BF2A68607870BB00BFD5F8DB
:1015900000C02968B1F850108C4421784FF006093A
:1015A00009EBC1010CF5806909EB4101084600BF58
:1015B000B0F80090C9F30909A0F800903E2E15D9A3
:1015C00000BF710906F01F09B9F1000F00D1491ED3
:1015D000B0F800904FF4004A4AEA812A1FFA8AFACA
:1015E00049EA0A09A0F800901BE01CE036B9B0F8FF
:1015F000009049F40049A0F8009012E000BF710883
:1016000006F00109B9F1000F00D0491CB0F80090B4
:101610004FF6FF7A0AEA812A49EA0A09A0F80090FF
:1016200000BF00BF0FE0607801280CD12868B0F837
:10163000500002442078062101EBC00002F58061D1
:1016400001EB40031E8000BFB3B200E004E06289FA
:101650006169286804F02FFD00BF227852002968D4
:1016600031F8121048F6BF7201EA020080F0100053
:1016700080F0200040F4004141F0800223785B00BC
:10168000296821F8132000BF0020BDE8F08702463A
:1016900001F0070000EB800302F5B47000EBC3001B
:1016A000C06970472DE9F04705460E4690461F4633
:1016B0004FF0000906F0800080280AD106F00700EC
:1016C00000EB800105F1280000EBC10401206070EF
:1016D00009E006F0070000EB800105F5B47000EBAF
:1016E000C1040020607006F007002070C4F810806C
:1016F000E770022F01D10020207100BF95F8A802E9
:10170000012802D10220BDE8F087012085F8A80257
:1017100000BF2146286803F00FFB00BF002085F8BA
:10172000A80200BF4846EEE72DE9F04105460E4607
:101730001746984606F0070000EB800105F5B470E7
:1017400000EBC1046761C4F818800020E06160709C
:1017500006F0070020702146286803F040FF0020B3
:10176000BDE8F08170B504460D4605F007006168DC
:10177000884201D9012070BD05F0800080280AD17F
:1017800005F0070000EB800104F1280000EBC10622
:101790000120707007E005EB850104F5B47000EBE3
:1017A000C106002070700120B07005F00700307095
:1017B00000BF94F8A802012801D10220DBE7012034
:1017C00084F8A80200BF3146206803F0DAFE05F075
:1017D000070020B904F52C71206803F062FE00BFF9
:1017E000002084F8A80200BF00BFC4E72DE9F04143
:1017F00005460E4690461F4606F0070000EB8001A6
:1018000005F1280000EBC104C4F81480A761012091
:1018100084F8240027620020E0610120607006F057
:10182000070020702146286803F0D9FE0020BDE89B
:10183000F0817FB50446206804F00AFC064606F4F1
:101840000040B0F5004F03D1204601F027FB7FBDDB
:1018500006F48060B0F5806F10D12068B0F84400C5
:101860004FF6FF3108402168A1F84400204600F0FF
:10187000B3F90021204600F0CFF9E8E706F48040F4
:10188000B0F5804F09D12068B0F844004BF6FF71E5
:1018900008402168A1F84400D9E706F40050B0F5EB
:1018A000005F09D12068B0F844004DF6FF71084090
:1018B0002168A1F84400CAE706F48050B0F5805FC3
:1018C0001ED12068B0F840004FF6FB710840216837
:1018D000A1F840002068B0F840004FF6F7710840CA
:1018E0002168A1F84000204600F088F92068B0F88F
:1018F00044004EF6FF7108402168A1F84400A6E7B5
:1019000006F40060B0F5006F56D1002507E06900CD
:10191000206830F811002DF81500681CC5B2082D9C
:10192000F5D32068B0F8400040F001002168A1F82C
:1019300040002068B0F840004FF6FE710840216872
:10194000A1F8400000BF2068B0F8440000F48060B7
:101950000028F8D02068B0F844004FF6FF31084066
:101960002168A1F84400002507E03DF815006A0051
:10197000216821F81200681CC5B2082DF5D3206833
:10198000B0F8400040F008002168A1F8400020684D
:10199000B0F844004FF2FF7108402168A1F84400FC
:1019A0002068B0F8400040F004002168A1F8400031
:1019B000204600F073F94AE706F40070B0F5007FA6
:1019C0000CD12068B0F844004FF6FF510840216860
:1019D000A1F84400204600F018F938E706F48070BA
:1019E000B0F5807F09D12068B0F844004FF6FF6160
:1019F00008402168A1F8440029E700BF27E730B577
:101A000085B0044614B9012005B030BD94F8A90290
:101A100028B9002084F8A802204600F095F8032099
:101A200084F8A902206803F032FD142204F11001A9
:101A30006846FEF779FB94E80F0003F0D5FB20B170
:101A4000022084F8A9020120DEE70021206804F0CA
:101A500028FB00252AE0012105EB850204F128007E
:101A600000EBC200417005EB850104F1280000F88D
:101A70003150002105EB850200EBC200C17005EB7F
:101A8000850204F1280000EBC200016105EB85022C
:101A900004F1280000EBC200416105EB850204F16E
:101AA000280000EBC2008161681CC5B26068A842D2
:101AB000D1D800252AE0002105EB850204F5B47099
:101AC00000EBC200417005EB850104F5B47000F82D
:101AD0003150002105EB850200EBC200C17005EB1F
:101AE000850204F5B47000EBC200016105EB8502CC
:101AF00004F5B47000EBC200416105EB850204F50A
:101B0000B47000EBC2008161681CC5B26068A84275
:101B1000D1D8142204F110016846FEF705FB94E8C1
:101B20000F0003F0A9FC20B1022084F8A9020120D3
:101B30006AE7002084F82400012084F8A9022068C4
:101B400003F097FC00205FE710B586B004461F49FC
:101B50002068884237D100BF1D48806940F00400EA
:101B60001B4988610846806900F00400019000BFAD
:101B700000BF00200290039004900590881402900A
:101B80000120039002200490059002A91148FEF75D
:101B900007FF0520FEF7F0FE00BF0D48C06940F4C6
:101BA00000000B49C8610846C06900F400000190BC
:101BB00000BF00BF002211461420FFF715F91420C2
:101BC000FFF702F900BF06B010BD0000005C004046
:101BD000001002400008014070B504460125A068CD
:101BE000022801D0FEF727FE2946D4F8EC0202F0C5
:101BF00079FDD4F8EC0202F02BFD70BD10B504465F
:101C0000D4F8EC0202F052FD10BD10B50446D4F831
:101C1000EC0202F056FD10BD70B504460D4600BF43
:101C200094F8A802012801D1022070BD012084F897
:101C3000A80200BF84F824502946206804F034FA32
:101C400000BF002084F8A80200BF00BFEDE710B578
:101C5000044604F52C71D4F8EC0202F05AFD10BDD4
:101C600010B5044600BF94F8A802012801D1022053
:101C700010BD012084F8A80200BF206804F0D7F945
:101C800001212046FFF724F9206803F0EFFB00BF95
:101C9000002084F8A80200BF00BFE9E710B50446A1
:101CA000D4F8EC0202F08EFDA06928B10348006868
:101CB00040F006000149086010BD000010ED00E092
:101CC000F8B5044600260025207800F00100002821
:101CD0006BD000274348C06900F0805070B900BF46
:101CE0004048C06940F080503E49C8610846C0691C
:101CF00000F08050009000BF00BF01273A48006804
:101D000000F48070B0B93848006840F480703649FB
:101D10000860FEF7E3FF064606E0FEF7DFFF801BE4
:101D2000642801D90320F8BD2F48006800F48070B2
:101D30000028F2D02B48006A00F440752DB3A0882B
:101D400000F44070A84220D02648006A20F4407574
:101D5000012026490860002008602248056205F03D
:101D6000010090B1FEF7BAFF064608E0FEF7B6FFA5
:101D7000801B41F28831884201D90320D3E71948FA
:101D8000006A00F002000028F0D01648006A20F433
:101D900040706168084313490862012F04D1084666
:101DA000C06920F08050C86100BF207800F00200B8
:101DB000022807D10B48406820F44040A16808433E
:101DC00008494860207800F01000102807D1054825
:101DD000406820F48000E168084302494860002020
:101DE000A1E70000001002400070004040044242A1
:101DF00070B504460D460CB9012070BD5A48006804
:101E000000F00700A8420ED25748006820F00700F3
:101E10002843554908600846006800F00700A842BA
:101E200001D00120E9E7207800F0020002281DD14E
:101E3000207800F00400042805D14C48406840F4A4
:101E4000E0604A494860207800F00800082805D181
:101E50004648406840F46050444948604348406800
:101E600020F0F000A168084340494860207800F065
:101E7000010078B36068012806D13C48006800F48E
:101E8000003090B90120B8E76068022806D13748D1
:101E9000006800F0007040B90120AEE733480068E8
:101EA00000F0020008B90120A7E73048406820F0A0
:101EB0000300616808432D494860FEF70FFF06469E
:101EC00009E0FEF70BFF801B41F28831884202D9FE
:101ED000032092E707E02548406800F00C006168A5
:101EE000B0EB810FEDD12048006800F00700A84258
:101EF0000ED91D48006820F0070028431A490860E1
:101F00000846006800F00700A84201D0012074E7ED
:101F1000207800F00400042807D11448406820F419
:101F2000E060E168084311494860207800F008004B
:101F3000082808D10D48406820F46050216940EA23
:101F4000C1000A49486000F03FF808494968C1F3F8
:101F50000311074A515CC8400649086006480068FA
:101F6000FEF7E2FE002048E7002002400010024099
:101F7000166A000878000020700000200148006800
:101F8000704700007800002000B5FFF7F7FF044914
:101F90004968C1F30221034A515CC84000BD0000FA
:101FA00000100240266A000800B5FFF7E7FF044969
:101FB0004968C1F3C221034A515CC84000BD00001A
:101FC00000100240266A000870B50021002200249B
:101FD00000230020134D696801F00C05F5B1042DB4
:101FE00002D0082D19D101E00F4819E00F4DC1F3BF
:101FF0008346AB5D01F4803555B10A4D6D68C5F37C
:1020000040450B4E725D084D5D43B5FBF2F402E0B6
:10201000084D03FB05F4204602E000BF024800BF64
:1020200000BF70BD0010024000127A00046A000870
:10203000146A000800093D00F8B504460CB90120F7
:10204000F8BD207800F00100002878D0F8484068FA
:1020500000F00C0004280CD0F548406800F00C009B
:10206000082811D1F248406800F48030B0F5803F74
:102070000AD1EF48006800F4003000285FD06068A3
:1020800000285CD10120DBE700BF6068B0F5803F2D
:1020900006D1E748006840F48030E549086028E050
:1020A000606858B9E248006820F48030E049086070
:1020B0000846006820F4802008601AE06068B0F5E7
:1020C000A02F0BD1DA48006840F48020D84908607E
:1020D0000846006840F4803008600AE0D448006890
:1020E00020F48030D24908600846006820F480203F
:1020F000086000BF606888B1FEF7F0FD054606E0A5
:10210000FEF7ECFD401B642801D9032098E7C8487E
:10211000006800F400300028F2D010E0FEF7DEFD89
:10212000054606E0FEF7DAFD401B642801D90320CE
:1021300086E7BF48006800F400300028F2D120781C
:1021400000F00200022857D1B948406800F00C00A6
:1021500050B1B748406800F00C00082818D1B448C6
:10216000406800F4803098B9B148006800F002007F
:1021700020B12069012801D0012061E7AC48006846
:1021800020F0F800616940EAC100A949086033E025
:102190002069E8B10120A7490860FEF79FFD0546C8
:1021A00006E0FEF79BFD401B022801D9032047E70C
:1021B0009F48006800F002000028F2D09C480068A8
:1021C00020F0F800616940EAC1009949086013E015
:1021D000002098490860FEF781FD054606E0FEF7FD
:1021E0007DFD401B022801D9032029E790480068A3
:1021F00000F002000028F2D1207800F00800082842
:102200002DD1A069B8B101208B490860FEF766FDA9
:10221000054606E0FEF762FD401B022801D90320B7
:102220000EE78348406A00F002000028F2D0012047
:1022300001F0AEF813E000207F490860FEF74EFD84
:10224000054606E0FEF74AFD401B022801D903209F
:10225000F6E67748406A00F002000028F2D12078C4
:1022600000F00400042873D100277148C06900F011
:10227000805070B900BF6E48C06940F080506C4912
:10228000C8610846C06900F08050009000BF00BFE0
:1022900001276A48006800F48070B0B96748006898
:1022A00040F4807065490860FEF718FD054606E0B9
:1022B000FEF714FD401B642801D90320C0E65F48E7
:1022C000006800F480700028F2D000BFE0680128A8
:1022D00006D15748006A40F001005549086227E0DE
:1022E000E06858B95248006A20F00100504908627D
:1022F0000846006A20F00400086219E0E06805283A
:102300000BD14B48006A40F0040049490862084676
:10231000006A40F0010008620AE04548006A20F0C7
:102320000100434908620846006A20F00400086280
:1023300000BFE068A0B1FEF7D1FC054609E0FEF75A
:10234000CDFC401B41F28831884202D9032077E658
:1023500022E03748006A00F002000028EFD012E0C7
:10236000FEF7BCFC054608E0FEF7B8FC401B41F256
:102370008831884201D9032062E62D48006A00F0C6
:1023800002000028F0D1012F05D12948C06920F0B2
:1023900080502749C86100BFE069C8B3244840683D
:1023A00000F00C00082860D0E069022848D1002025
:1023B00020490866FEF792FC054606E0FEF78EFC13
:1023C000401B022801D903203AE61948006800F0B2
:1023D00000700028F2D1206AB0F5803F07D1144880
:1023E000406820F40030A168084311494860D4E9EE
:1023F000080108430E49496821F4741108430C4947
:10240000486001200B490866FEF768FC054607E0B6
:102410003DE0FEF763FC401B022801D903200FE6D4
:102420000348006800F000700028F2D02FE00000A0
:10243000001002400000424280044242007000400E
:10244000002014490866FEF749FC054606E0FEF741
:1024500045FC401B022801D90320F1E50E48006825
:1024600000F000700028F2D111E0E069012800D1ED
:10247000E6E50948466806F48031206A814204D1C5
:1024800006F47011606A814201D00120D8E5002075
:10249000D6E50000000042420010024070B504463C
:1024A0002546681EB0F1807F01D301200FE0681E31
:1024B0004FF0E02148610F214FF0FF3003F026FE7E
:1024C00000204FF0E021886107200861002070BDE6
:1024D00030B502460B4600BF92F83C00012801D1FE
:1024E000022030BD012082F83C0000BF022082F8AB
:1024F0003D00106844681068816824F07004186812
:10250000044310684460104D1068A8420BD0106856
:10251000B0F1804F07D00D4D1068A84203D00C4D8C
:102520001068A84205D121F0800158680143106865
:102530008160012082F83D0000BF002082F83C004D
:1025400000BF00BFCDE70000002C014000040040A8
:102550000008004010B586B00446002002900390A9
:10256000049005902068B0F1804F21D100BF114840
:10257000806940F008000F4988610846806900F0D2
:102580000800019000BF00BF0820029002200390C5
:10259000059002A90848FEF703FA00BF07494868FA
:1025A00020F4407040F0E06040F48070486000BF6C
:1025B00006B010BD00100240000C014000000140B8
:1025C0002DE9F04104460D461646002700BF94F859
:1025D0003C00012802D10220BDE8F081012084F8EE
:1025E0003C0000BF36B1042E1BD0082E31D00C2E7B
:1025F0005ED145E02946206800F064FF20688069CC
:1026000040F00800216888612068806920F004009B
:102610002168886120688069296908432168886188
:1026200048E02946206800F07DFF2068806940F47A
:102630000060216888612068806920F480602168DA
:10264000886120688069296940EA012021688861E1
:1026500030E02946206800F099FF2068C06940F00A
:1026600008002168C8612068C06920F00400216862
:10267000C8612068C069296908432168C86119E0F8
:102680002946206800F0B6FF2068C06940F4006069
:102690002168C8612068C06920F480602168C86131
:1026A0002068C069296940EA01202168C86101E009
:1026B000012700BF00BF00BF002084F83C0000BF1E
:1026C000384689E710B504460CB9012010BD94F8CE
:1026D0003D0028B9002084F83C00204600F026F890
:1026E000022084F83D00211D206800F0B1FE012089
:1026F00084F8460000BF84F83E0001213F200155C8
:10270000402001554120015500BF00BF012084F841
:10271000420043200155442001554520015500BF8A
:10272000012084F83D000020D0E7000008B50168D2
:10273000B1F1804F0DD100BF0649C96941F00101D7
:10274000044AD1611146C96901F00101009100BF3D
:1027500000BF08BD00100240704770472DE9F84FD8
:102760000446206805682068C668206847694FF0FD
:102770000009CA4605F00F09B9F1000F0AD105F0AA
:10278000200038B106F0200020B1204600F0A6FF5E
:10279000BDE8F88FB9F1000F7BD007F0010018B940
:1027A00006F49070002874D005F0010030B106F4F2
:1027B000807018B1606C40F00100606405F00400A6
:1027C00030B107F0010018B1606C40F002006064A5
:1027D00005F0020030B107F0010018B1606C40F064
:1027E0000400606405F0080048B106F0200010B94C
:1027F00007F0010018B1606C40F008006064606C84
:10280000002845D005F0200028B106F0200010B1C6
:10281000204600F063FF20684069C0F3801A606CB6
:1028200000F0080010B9BAF1000F2CD0204600F0DB
:102830000FFF2068406900F0400000B300BF00BFF8
:102840002168143151E8001F21F040002168143143
:1028500041E80002002AF3D100BFE06B50B1774895
:10286000E16B4863E06BFEF72FF888B1E06B416BDA
:1028700088470DE02046FFF770FF09E009E0204699
:10288000FFF76BFF04E02046FFF767FF002060645E
:102890007EE7206B012877D105F01000002873D067
:1028A00006F010000028FAD000BF00200090206839
:1028B0000068009020684068009000BF00BF20685A
:1028C000406900F0400000285FD0E06B006840687D
:1028D0001FFA80F8B8F1000F55D0A08D404552DDA9
:1028E000A4F82E80E06B8069202843D000BF00BF91
:1028F00021680C3151E8001F21F4807021680C31EF
:1029000041E80002002AF3D100BF00BF00BF2168E8
:10291000143151E8001F21F001002168143141E811
:102920000002002AF3D100BF00BF00BF21681431AC
:1029300051E8001F21F040002168143141E80002F5
:10294000002AF3D100BF202084F842000020206339
:1029500000BF00BF21680C3151E8001F21F01000BA
:1029600021680C3141E80002002AF3D100BFE06B7E
:10297000FDF77EFF02206063A08DE28D801A81B298
:102980002046FFF7E9FE03E742E0A08DE18D401A03
:102990001FFA80F8E08DD0B3B8F1000F37D000BF38
:1029A00000BF21680C3151E8001F21F490702168AC
:1029B0000C3141E80002002AF3D100BF00BF00BF84
:1029C0002168143151E8001F21F001002168143101
:1029D00041E80002002AF3D100BF202084F8420021
:1029E0000020206300BF00BF21680C3151E8001FA8
:1029F00021F0100021680C3141E80002002AF3D1D7
:102A000000BF0220606341462046FFF7A5FEBFE6F7
:102A100005F0800030B106F0800018B1204600F0CB
:102A200079FFB5E605F0400030B106F0400018B17E
:102A3000204600F043FEABE600BFA9E63D360008A5
:102A400010B504460CB9012010BDA06900B100E02A
:102A500000BF94F8410028B9002084F840002046C7
:102A600000F02AF8242084F841002068C06820F48F
:102A700000502168C860204600F0AEFE2068006962
:102A800020F49040216808612068406920F02A0005
:102A9000216848612068C06840F400502168C8601F
:102AA00000206064202084F8410084F84200002067
:102AB000606300BFC8E7000010B586B00446002080
:102AC00002900390049005901E492068884236D1F8
:102AD00000BF1D48806940F480401B49886108465A
:102AE000806900F48040019000BF00BF00BF08462D
:102AF000806940F0040088610846806900F00400A5
:102B0000019000BF00BF48150290022003900320EF
:102B1000059002A90D48FDF743FF4FF48060029035
:102B200000200390049002A90848FDF739FF002215
:102B300011462520FEF758F92520FEF745F906B085
:102B400010BD0000003801400010024000080140A4
:102B500070B504460D46164694F8420020280BD165
:102B600005B10EB9012070BD002020633246294610
:102B7000204600F0AFFEF6E70220F4E710B5044669
:102B800003492068884201D103F05EFD10BD0000BA
:102B9000003801402DE9F84F04460E461746994685
:102BA0004FF0000A94F8410020284AD106B117B925
:102BB0000120BDE8F88F00206064212084F84100E6
:102BC000FEF78CF88246A784E784A068B0F5805FA2
:102BD00004D1206910B90025B04602E035464FF017
:102BE00000081BE05346002280212046CDF80090CB
:102BF00000F0C0FE08B10320DBE745B9B8F80000DB
:102C0000C0F308002168486008F1020803E0287852
:102C1000216848606D1CE08C401EE084E08C002838
:102C2000E0D15346002240212046CDF8009000F02C
:102C3000A1FE08B10320BCE7202084F84100002059
:102C4000B7E70220B5E7704700BFFEE730B50B4697
:102C5000002100BF16E00A24B4EB107F05D9302410
:102C600004EB107403F8114005E0412404EB1074E8
:102C70000A3C03F81140000100254C00641C1D555E
:102C80004C1CE1B29142E6DB30BD000000B585B0DE
:102C90000020019002900390049000BF39488069A1
:102CA00040F01000374988610846806900F0100044
:102CB000009000BF00BF00BF0846806940F02000C0
:102CC00088610846806900F02000009000BF00BFC6
:102CD00000BF0846806940F00400886108468069AA
:102CE00000F00400009000BF00BF00BF08468069EC
:102CF00040F0080088610846806900F008000090F4
:102D000000BF00BF012248F288011F48FDF7E0FF25
:102D1000012241211D48FDF7DBFF002220211B4835
:102D2000FDF7D6FF48F288000190012002900020B4
:102D300003900220049001A91348FDF731FE6120A1
:102D4000019001200290002003900220049001A92C
:102D50000E48FDF725FE0220019000200290012080
:102D6000039001A90948FDF71BFE4FF42470019060
:102D700000200290039001A90448FDF711FE05B060
:102D800000BD00000010024000080140000C01409E
:102D900000B589B00020079008901C216846FDF717
:102DA000DCF94FF080401849086047204860002156
:102DB0001548816040F22B11C16000210161802122
:102DC0008161FFF77FFC08B1FDF735FD002007901A
:102DD000089007A90C48FFF77BFB08B1FDF72BFD16
:102DE0006020009095200190002002900490042221
:102DF00069460548FFF7E4FB08B1FDF71CFD0248F2
:102E0000FFF7A8FB09B000BDC401002010B50B48B6
:102E10000B4908604FF41650486000210848816053
:102E2000C16001610C21416100218161C161FFF735
:102E300007FE08B1FDF7FFFC10BD0000003801409F
:102E40000C02002010B503F06FFA00220D490E4865
:102E500001F055FA08B1FDF7EEFC0C490A4801F003
:102E6000E7FC08B1FDF7E7FC0949074800F005FF5A
:102E700008B1FDF7E0FC044801F0A4FD08B1FDF73E
:102E8000DAFC10BD080000207C0200208C0000202D
:102E90005C00002000BFFEE700BFFEE72DE9F05F09
:102EA00005466AE22868B0F844A00AF00F07002F30
:102EB0007DD10AF01000B0BB00BF2968098848F630
:102EC0000F7201EA020040F400412A68118000BF3D
:102ED00005F128042868B0F85010207801EBC000F4
:102EE000801C296801F5806131F81000C0F30900E9
:102EF000E061E16960690844606100212846FDF7EE
:102F0000E8FF95F824000028CBD0A0690028C8D19C
:102F100095F8240040F080002968A1F84C000020BA
:102F200085F8240029E2FFE705F5B47428680688CF
:102F300006F4006030B32868B0F85010207801EB38
:102F4000C000801D296801F5806131F81000C0F3D0
:102F50000900E061A18B8BB2E28805F52C7128682D
:102F600003F07AF800BF2968098840F68F7201EAF9
:102F7000020040F080012A68118000BF2846FEF759
:102F800066FEFAE106F4004000288AD000BF2968F6
:102F9000098840F68F7201EA020040F080012A6839
:102FA000118000BF2868B0F85010207800E07AE067
:102FB00001EBC000801D296801F5806131F8100027
:102FC000C0F30900E061E06990B1606980B1B4F8D4
:102FD0001CC01FFA8CF3E2886169286803F03CF892
:102FE000E16960690844606100212846FDF781FFBE
:102FF0002868068806F40060002893D106F4405043
:10300000B0F5405F8ED000BF2A682968B1F8501033
:103010000A4402F20C41084600BF0388C3F30903C7
:10302000038023693E2B12D900BF23695909237CF1
:1030300003F01F0303B9491E03884FF4004C4CEA08
:10304000812C1FFA8CFC43EA0C03038017E02369F0
:1030500023B9038843F40043038010E000BF2369D1
:103060005908237C03F0010303B1491C03884FF680
:10307000FF7C0CEA812C43EA0C03038000BF00BFF5
:1030800000BF00BF296809884BF68F7201EA020071
:1030900080F4805080F4005040F4004141F0800101
:1030A0002A68118069E17900286830F8116006F417
:1030B000004000286FD000BF7A00296831F8121054
:1030C00040F68F7201EA020040F080017B002A681E
:1030D00022F8131000BF07EB870105F5B47000EB71
:1030E000C104207BB8B92868B0F85010207801EBF3
:1030F000C000801D296801F5806131F81000C0F31F
:103100000908B8F1000F5ED0E2886169434628687B
:1031100002F0A2FF57E0E078022806D132462146AD
:103120002846FDF769FF80464DE000BF00BF2278CA
:103130005200296831F8121048F68F7201EA020035
:1031400040F4004141F0C00123785B002A6822F876
:10315000131000BF00BF21784900286830F8110023
:1031600000F48040C0B12868B0F85010207801EB1E
:10317000C000801C296801F5806131F81000C0F39F
:103180000908B8F1000F1ED02289616943462868FA
:1031900002F062FF17E02AE02868B0F850102078AB
:1031A00001EBC000801D296801F5806131F8100035
:1031B000C0F30908B8F1000F05D062896169434680
:1031C000286802F049FFE0694044E06160694044DA
:1031D0006061A06910B12069404504D92178284672
:1031E000FDF787FE03E02146286802F0F8F906F0B3
:1031F0008000002876D007EB870105F1280000EB5E
:10320000C10400BF7A00296831F8121048F60F7225
:1032100001EA020040F400417B002A6822F8131002
:1032200000BFE078012876D10020A061207B002833
:103230006BD006F0400080B300BF6078C0B900BF1B
:1032400029682A68B2F8502011442278022303EB3F
:10325000C20201F5806303EB420000BF0288C2F3A3
:1032600009020280028842F40042028000BF13E09B
:103270006078012810D100BF28682A68B2F8502071
:1032800010442278022303EBC20200F5806303EBB3
:10329000420100220A8000BF37E0FFE700BF296833
:1032A000607800BB00BF2B68D5F800C0BCF850C0E8
:1032B000634494F800C04FF0060B0BEBCC0C03F505
:1032C000806B0BEB4C0000BFB0F800C0CCF3090CD6
:1032D000A0F800C0B0F800C04CF4004CA0F800C04A
:1032E00000BF11E049E0607801280DD12868B0F8EE
:1032F000500001442078062303EBC00001F58063F1
:1033000003EB40020020108000BF21782846FDF723
:10331000E0FD32E0FFE706F4807048BB2868B0F8B3
:103320005010207801EBC000801C296801F58061F5
:1033300031F81000C0F30909A069484504D9A06913
:10334000A0EB0900A06101E00020A061A06920B904
:1033500021782846FDF7BDFD0FE0606948446061B3
:10336000E0694844E0612146286802F038F904E049
:10337000324621462846FDF7EBFE2868B0F84400A7
:1033800000F4004000287FF48DADBDE8F09F704749
:1033900008B508490968C9084FF47A72B1FBF2F11F
:1033A0004143009100BF00BF00994A1E00920029CE
:1033B000F9D108BD78000020704710B502F0F4FF85
:1033C00003F0E6FAFDF790FC10BD00B593B028219C
:1033D00009A8FCF7C2FE142104A8FCF7BEFE0020D9
:1033E00000900190029003900120099000040A903F
:1033F00000200B9001200D9002201090C10311912C
:103400004FF4E011129109A8FEF716FE08B1FDF77E
:1034100012FA0F20049002200590002006904FF42D
:103420008060079000200890022104A8FEF7E0FCCD
:1034300008B1FDF700FA10200090002003906846C4
:10344000FEF73EFC08B1FDF7F6F913B000BD70477A
:1034500010B50268184B984208D0B0F1804F05D0E3
:10346000164B984202D0164B984203D122F07002BC
:103470004B681A43104B984208D0B0F1804F05D0EA
:103480000E4B984202D00E4B984203D122F4407268
:10349000CB681A4322F080034C6943EA04020260BD
:1034A0008B68C3620B688362034B984201D10B693E
:1034B00003630123436110BD002C01400004004060
:1034C0000008004030B5026A056A25F00105056272
:1034D0004368846924F0700424F003040D682C43CD
:1034E00022F002028D682A430D4DA84206D100BF8A
:1034F00022F00802CD682A4322F00402084DA842B7
:1035000007D123F4807323F400734D692B438D6935
:103510002B43436084614D684563026230BD000007
:10352000002C014030B5026A056A25F010050562DD
:103530004368846924F4E04424F440740D6844EA48
:10354000052422F020028D6842EA05120E4DA842A1
:1035500007D100BF22F08002CD6842EA051222F0B6
:103560004002094DA84209D123F4806323F400638B
:103570004D6943EA85038D6943EA850343608461AD
:103580004D688563026230BD002C014030B5026A8F
:10359000056A25F4807505624368C46924F07004E7
:1035A00024F003040D682C4322F400728D6842EA73
:1035B00005220F4DA84207D100BF22F40062CD685A
:1035C00042EA052222F48062094DA84209D123F47F
:1035D000805323F400534D6943EA05138D6943EA90
:1035E00005134360C4614D68C563026230BD0000CD
:1035F000002C014030B5036A056A25F48055056248
:103600004468C26922F4E04222F440720D6842EA42
:10361000052223F400538D6843EA0533064DA84282
:1036200004D124F480444D6944EA85144460C261A5
:103630004D680564036230BD002C014070B505463D
:103640006C6A0020E085E0842046FFF786F870BDB4
:1036500000BF00BF02680C3252E8002F22F49071C4
:1036600002680C3242E80013002BF3D100BF00BF08
:1036700000BF0268143252E8002F22F001010268F4
:10368000143242E80013002BF3D100BF016B012973
:103690000ED100BF00BF02680C3252E8002F22F0AA
:1036A000100102680C3242E80013002BF3D100BF76
:1036B000202180F8421000210163704710B50446B4
:1036C0002068C06820F040002168C860202084F88D
:1036D00041002046FFF7B7FA002010BDF8B50446B8
:1036E00094F84200222875D1A068B0F5805F0CD113
:1036F000206950B90025A66A20684068C0F3080018
:103700003080A06A801CA06215E0A56A0026A0682F
:10371000B0F5805F03D0A06828B9206918B9206887
:103720004068287004E02068406800F07F0028703E
:10373000A06A401CA062E08D401E80B2E085002897
:1037400046D12068C06820F020002168C860206849
:10375000C06820F480702168C8602068406920F04B
:10376000010021684861202084F842000020606345
:10377000206B012826D10020206300BF00BF2168F4
:103780000C3151E8001F21F0100021680C3141E894
:103790000002002AF3D100BF2068006800F010008A
:1037A00010280AD100BF0020009020680068009017
:1037B00020684068009000BF00BFA18D2046FEF742
:1037C000CBFF02E02046FFF7D9F90020F8BD01E069
:1037D0000020FBE70220F9E770B50446216809697B
:1037E00021F44051E2681143226811612269A16805
:1037F0001143626941EA02052168C96841F20C621D
:10380000914329432268D1602168496921F44071BC
:10381000A2691143226851612D4A2168914202D167
:10382000FEF7C2FB01E0FEF7AFFB00EBC00101EBCE
:10383000001162689200B1FBF2F100EBC00202EBF2
:10384000001263689B00B2FBF3F26423B2FBF3F255
:1038500002EBC20303EB0212A1EB8201322202EB64
:1038600001116422B1FBF2F101F0F00100EBC002A2
:1038700002EB001263689B00B2FBF3F26423B2FB1D
:10388000F3F201EB021200EBC00101EB00116368DF
:103890009B00B1FBF3F100EBC00303EB0013666880
:1038A000B600B3FBF6F36426B3FBF6F303EBC306F3
:1038B00006EB0313A1EB8301322303EB0111642315
:1038C000B1FBF3F101F00F0111442268916070BD6A
:1038D0000038014010B5034699629A85DA850020C8
:1038E0005864222083F84200186928B11868C0681B
:1038F00040F480701C68E0601868406940F0010086
:103900001C6860611868C06840F020001C68E060B6
:10391000002010BD014691F84100212828D1886877
:10392000B0F5805F0BD1086948B90A6A1088C0F306
:1039300008000B685860086A801C086205E00B6A82
:10394000581C086218780B685860C88C401E80B2FA
:10395000C88458B90868C06820F080000B68D86037
:103960000868C06840F040000B68D86000207047CD
:103970000220FCE72DE9F04104460D461746984623
:10398000069E34E0701C88B32EB1FDF7A7F9A0EBBA
:103990000800B0422BD900BF00BF21680C3151E8AC
:1039A000001F21F4D07021680C3141E80002002A88
:1039B000F3D100BF00BF00BF2168143151E8001FE0
:1039C00021F001002168143141E80002002AF3D1FE
:1039D00000BF202084F8410084F8420000BF00208E
:1039E00084F8400000BF0320BDE8F081FFE72068B5
:1039F00000682840A84201D1012000E00020B84220
:103A0000C0D00020F0E7000010B50248FEF7A6FE87
:103A100010BD00000C0200202DE9F04104460D46C7
:103A2000D4F8B862D4F8C072D4F8B80278B305EB11
:103A3000850104F1140000EB8100806808B305EBF8
:103A4000850104F1140000EB810005EB850281681B
:103A500007F1280000EBC2000069B1FBF0F200FBA7
:103A6000121070B9002105EB850204F1140000EB7F
:103A70008200816000231A462946204600F0ACFEF1
:103A800002E00020C6F814020020BDE8F081FFE744
:103A90000220FAE770B504460E46D4F8B852314613
:103AA000204600F03EFDC5F80C02D4F8B80248B13B
:103AB000D5F80402D4F8BC12CA6805F50371904722
:103AC000002070BD0220FCE770B504460E460025BC
:103AD0008121204600F03FFC0021E16201212046C7
:103AE00000F039FC0021C4F86C118221204600F05E
:103AF00032FC00212164D4F8B80250B1D4F8BC12D1
:103B000048688047D4F8B80201F00FF90020C4F8E3
:103B1000B802284670BD70B50546D5F8B842D5F84C
:103B2000BC0278B194F80002FF280BD094F801226F
:103B300094F80002D5F8BC128B6821469847FF2004
:103B400084F80002002070BD01460A200880014868
:103B50007047000080000020014643200880014893
:103B600070470000080100200146432008800148FA
:103B700070470000C400002001464320088001482F
:103B8000704700004C0100202DE9F04104460F462B
:103B90000026207C88B94FF4007302228121204640
:103BA00000F026FD0121E1624B020222204600F0D6
:103BB0001FFD0121C4F86C110FE040230222812176
:103BC000204600F015FD0121E1624023022220463B
:103BD00000F00EFD0121C4F86C110823032282219C
:103BE000204600F005FD012121644FF4077001F02B
:103BF0009DF8C4F8B802D4F8B80208B901261CE050
:103C0000D4F8B852D4F8BC12086880470020C5F830
:103C10001402C5F81802207C40B94FF4007301214A
:103C20002046D5F8042200F0FBFC06E040230121E9
:103C30002046D5F8042200F0F3FC3046BDE8F081C0
:103C400070B50446D4F8B852D4F8B80298B1207CC4
:103C500040B94FF4007301212046D5F8042200F04A
:103C6000DFFC06E0402301212046D5F8042200F0C5
:103C7000D7FC002070BD0220FCE70246022011B1F3
:103C8000C2F8BC12002070470246D2F8B832C3F81E
:103C900004120020704710B50346D3F8B842C4F8A8
:103CA0000812C4F81022002010BD2DE9FC41054681
:103CB0000C46D5F8B86200200190009000272078CB
:103CC00000F0600040B320285FD1E088E0B12078A8
:103CD00000F0800060B1E2886078D5F8BC128B6893
:103CE00031469847E2883146284600F0C7F812E08E
:103CF000607886F80002A07986F80102E2883146F1
:103D0000284600F09AF806E06078D5F8BC12002248
:103D10008B68214698473EE0607820B10A2812D08F
:103D20000B282AD11FE095F89C02032805D1022216
:103D30006946284600F0A2F804E02146284600F033
:103D400070F802271FE095F89C02032805D1012294
:103D500001A9284600F092F804E02146284600F028
:103D600060F802270FE095F89C02032804D0214652
:103D7000284600F056F8022705E02146284600F0C4
:103D800050F8022700BF00BF05E02146284600F09A
:103D900048F8022700BF00BF3846BDE8FC8170B577
:103DA00004460D46D4F8B40229464268204690479E
:103DB000002070BD70B504460D4694F89C020128A1
:103DC00004D0022803D003280CD101E000BF00BFBB
:103DD0006888012805D10020C4F8A402204600F01C
:103DE0005EF804E02946204600F01BF800BF00BF43
:103DF00070BD70B506460C4615462B46224600217E
:103E0000304600F00DFC002070BD70B506460C4633
:103E100015462B4622460021304600F0DDFC0020EE
:103E200070BD70B504460D468021204600F0A8FC08
:103E30000021204600F0A4FC70BD70B504460E467B
:103E400015460320C4F894024FF4AE700551001DCE
:103E500005512B4632460021204600F0E1FB0020B0
:103E600070BD10B504460520C4F8940200231A461C
:103E70001946204600F0D4FB002010BD70B5044662
:103E80000E4615460220C4F89402E56125622B46D1
:103E900032460021204600F09FFC002070BD10B586
:103EA00004460420C4F8940200231A46194620460A
:103EB00000F092FC002010BD70B505460C462DB9EF
:103EC0002246064906A000F0DBF904E02246034939
:103ED00003A000F0D5F9014870BD000040050020A6
:103EE00043444320436F6E66696700000246122018
:103EF00008800148704700002400002070B5054686
:103F00000C462DB92246064906A000F0B9F904E096
:103F10002246034903A000F0B3F9014870BD000038
:103F20004005002043444320496E74657266616316
:103F30006500000002460420088001487047000028
:103F40003800002070B505460C462246024903A001
:103F500000F096F9004870BD4005002053544D69AB
:103F600063726F656C656374726F6E696373000072
:103F700070B505460C462DB92246064906A000F04C
:103F80007FF904E02246034903A000F079F90148D3
:103F900070BD00004005002053544D333220566957
:103FA000727475616C20436F6D506F727400000005
:103FB00070B505460C461A202080FCF73FFC0148EE
:103FC00070BD00003C00002070B504460D46E88836
:103FD000012804D029462046FFF723FF1EE094F86D
:103FE0009C02012804D0022803D0032810D109E044
:103FF00000BF0020A060012204F108012046FFF765
:104000003DFF0AE00122211D2046FFF737FF04E0B3
:1040100029462046FFF705FF00BF00BF70BDF8B579
:1040200004460E46002000900027002570880012EC
:10403000082875D2DFE800F0C7040C20C7C7A5B573
:10404000207CD4F8B0120A68694690470746C1E060
:10405000207C40B9D4F8B402816A68468847074694
:104060000220787007E0D4F8B402C16A6846884735
:10407000074602207870ADE0B078062878D2DFE8F5
:1040800000F00316293C5063D4F8B002406838B100
:10409000207CD4F8B0124A6869469047074605E08C
:1040A00031462046FFF7BDFE681CC5B267E0D4F874
:1040B000B002806838B1207CD4F8B0128A686946B2
:1040C0009047074605E031462046FFF7AAFE681CE8
:1040D000C5B254E0D4F8B002C06838B1207CD4F83E
:1040E000B012CA6869469047074605E03146204647
:1040F000FFF797FE681CC5B241E0D4F8B002006932
:1041000038B1207CD4F8B0120A6969469047074656
:1041100005E031462046FFF784FE681CC5B22EE05C
:1041200051E0D4F8B002406938B1207CD4F8B01224
:104130004A6969469047074605E031462046FFF741
:1041400070FE681CC5B21AE0D4F8B002806940B1B4
:10415000207CD4F8B0128A6969469047074606E089
:1041600006E031462046FFF75CFE681CC5B206E05B
:1041700031462046FFF755FE681CC5B200BF00BFA0
:1041800028E0207C30B9D4F8B402416B68468847F7
:10419000074605E031462046FFF743FE681CC5B2DE
:1041A00018E0207C40B9D4F8B402016B6846884717
:1041B00007460720787005E031462046FFF731FEBC
:1041C000681CC5B206E031462046FFF72AFE681C8F
:1041D000C5B200BF00BF05B1F8BDBDF8000088B191
:1041E000F08878B1F088BDF80010884202DDBDF893
:1041F000000000E0F0880090BDF80020394620461D
:10420000FFF73CFEF08810B92046FFF748FE00BFDC
:10421000E2E70146002002E0421CD0B2491C0A78C5
:10422000002AF9D1704770B504460D4694F89C02F7
:10423000012804D0022803D003281AD101E000BFCE
:1042400000BFE888022804D029462046FFF7E9FD90
:1042500014E00120E060D4F8A40218B1E06840F056
:104260000200E060022204F10C012046FFF706FE86
:1042700004E029462046FFF7D4FD00BF00BF70BD13
:104280002DE9F04104460D4617460026FCB12046B4
:10429000FFF7BFFF022101EB400038803A7830463B
:1042A000711CCEB22A5403223046711CCEB22A545D
:1042B0000AE014F8012B3046711CCEB22A540022B9
:1042C0003046711CCEB22A5420780028F1D1BDE8C6
:1042D000F0810146002031B1012906D0022906D023
:1042E000032908D105E0002007E0022005E00120B5
:1042F00003E0022001E0022000BF00BF704770B55C
:1043000004460D4616460CB9022070BDD4F8B4021E
:1043100010B10020C4F8B4020DB1C4F8B0520120AD
:1043200084F89C022670204600F004F90020ECE797
:104330002DE9F04104460D46002600272946D4F811
:10434000C002FCF71BFE06463046FFF7C2FF0746D9
:104350003846BDE8F0812DE9F04104460D460026BF
:1043600000272946D4F8C002FCF7D3FD06463046A4
:10437000FFF7AFFF07463846BDE8F0812DE9F04171
:1043800004460E461746002E64D104F11405D4F8F5
:104390009402022848D1D5E90301884210D9D5E911
:1043A0000301401AE860A88982B239462046FFF727
:1043B0002CFD00231A461946204600F031F93EE054
:1043C0002969A868B0FBF1F201FB1200B8B92969AC
:1043D000A868884213D3A868D4F8981288420ED2ED
:1043E000002211462046FFF710FD0020C4F8980275
:1043F00000231A461946204600F012F91FE0D4F8AF
:10440000B402C06840B194F89C02032804D1D4F8E7
:10441000B402C168204688478021204600F0B0F9E8
:104420002046FFF71EFD0AE0D4F89402042802D0CB
:10443000D4F8940218B98021204600F0A1F994F82C
:10444000A002012818D1204600F0FAF9002084F8D3
:10445000A00211E0D4F8B402406950B194F89C0273
:10446000032806D1D4F8B402314642692046904769
:1044700002E00220BDE8F0810020FBE72DE9F041D9
:1044800004460E461746BEBB04F5AA75D4F894023E
:10449000032825D1D5E90301884210D9D5E90301C4
:1044A000401AE860D5E90301884201D2E86800E0DB
:1044B000286982B239462046FFF79BFC2FE0D4F8EA
:1044C000B402006940B194F89C02032804D1D4F8E6
:1044D000B4020169204688472046FFF7E0FC1EE051
:1044E000D4F8940205281AD10020C4F894020021BF
:1044F000204600F045F912E0FFE7D4F8B4028069E5
:1045000050B194F89C02032806D1D4F8B402314685
:1045100082692046904702E00220BDE8F081002039
:10452000FBE770B504460D462946D4F8C002FDF7F6
:10453000AEF870BD10B504461D48C0F8EC42C4F892
:10454000C0021C481A490860082048600221184827
:10455000816000218161C1610162FDF750FA08B1FB
:10456000FCF769F904F5307418230022114620681D
:10457000FCF78CFC5823002280212068FCF786FC85
:10458000C023002281212068FCF780FC4FF488734F
:10459000002201212068FCF779FC2068A4F5307422
:1045A0004FF4807300228221FCF770FC002010BDC4
:1045B00040110020005C004010B50246D2F8C03225
:1045C00001F08000802809D101F07F0000EB800419
:1045D00003F1280000EBC400807810BD01F07F00DB
:1045E00000EB800403F5B47000EBC4008078F4E7BE
:1045F0002DE9F04704460F4615461E464FF00008C9
:10460000C1462B4632463946D4F8C002FDF74AF877
:1046100080464046FFF75DFE81464846BDE8F0878C
:104620002DE9F04704460D4616461F464FF0000898
:10463000C1463B4632462946D4F8C002FDF774F81D
:1046400080464046FFF745FE81464846BDE8F08774
:1046500010B504464023002211462046FFF7C8FF4C
:1046600001214FF4AC70015140214FF4B27001515F
:104670004023002280212046FFF7BAFF0121A161DB
:1046800040216162012084F89C020020C4F8940259
:104690006060C4F8A402D4F8B80228B12179D4F833
:1046A000B402426820469047002010BD014691F8B0
:1046B0009C02042803D191F89D0281F89C020020FD
:1046C000704710B5044694F89C02032808D1D4F82A
:1046D000B402C06920B1D4F8B402C1692046884749
:1046E000002010BD02461174002070472DE9F041F2
:1046F00004460D46002600272946D4F8C002FDF7DF
:104700008BFA06463046FFF7E4FD07463846BDE81B
:10471000F08170B504460D46294604F52A7000F074
:1047200073F80120C4F8940240F2AE20005BC4F894
:10473000980294F8A80200F01F0020B1012808D0C8
:10474000022812D10BE004F52A71204600F041F94D
:1047500013E004F52A71204600F0A8FA0DE004F5F4
:104760002A71204600F086F907E094F8A80200F0CC
:104770008001204600F004F800BF00BF002070BD9B
:104780002DE9F04104460D46002600272946D4F8BD
:10479000C002FCF7E7FF06463046FFF79AFD0746E2
:1047A0003846BDE8F08170B5044600250026D4F8EF
:1047B000C002FDF755FA05462846FFF78AFD064672
:1047C000304670BD014691F89C0281F89D0204209C
:1047D00081F89C02002070472DE9F04704460D4601
:1047E00016461F464FF00008C1463B463246294652
:1047F000D4F8C002FCF7FAFF80464046FFF769FD97
:1048000081464846BDE8F0870A7802704A784270CF
:104810008B78CA7803EB022242800B794A7903EB4A
:10482000022282808B79CA7903EB0222C280704710
:104830000246002011B1C2F8B41200E00220704715
:1048400001460020704770B504460D46A88810BB8D
:10485000E88800BB688880281DD2A87800F07F0611
:1048600094F89C02032804D129462046FFF7D9FA80
:1048700015E084F89E6231462046FFF737FF204658
:10488000FFF70DFB1EB1022084F89C0207E0012017
:1048900084F89C0203E029462046FFF7C2FA70BD67
:1048A00070B504460D460226D4F8B40238B1D4F8E7
:1048B000B402294602682046904700B900263046D7
:1048C00070BD000070B504460D46A87836490870E2
:1048D00008460078012804DD29462046FFF7A1FAA2
:1048E00060E094F89C02022802D003284FD11CE01B
:1048F0002D480078A8B12C4800786060032084F827
:104900009C02294801782046FFF7CAFF022804D1FB
:1049100029462046FFF785FA70BD2046FFF7BFFA0B
:1049200002E02046FFF7BBFA3BE01F48007870B971
:10493000022084F89C021C48007860601A480178C4
:104940002046FFF72CFA2046FFF7A9FA1EE0164989
:1049500009786068884216D021792046FFF71FFA4F
:10496000114800786060104801782046FFF798FFF2
:10497000022804D129462046FFF753FACCE7204607
:10498000FFF78DFA02E02046FFF789FA09E0294691
:104990002046FFF746FA044801782046FFF7FFF962
:1049A00000BF00BF00BFB7E77C00002070B5054620
:1049B0000C466088012804D1C5F8A4022846FFF7F8
:1049C0006EFA70BD10B504462046FFF7ECFE0020DD
:1049D00010BD70B505460C460026207800F060003A
:1049E00060B1202802D040283CD100E000BFD5F8BB
:1049F000B402214682682846904738E060780A2849
:104A000029D2DFE800F01923281E280A0528140FF0
:104A100021462846FFF703FB22E021462846FFF700
:104A200012FF1DE021462846FFF74CFF18E0214603
:104A30002846FFF7C9FA13E021462846FFF7F3FBA3
:104A40000EE021462846FFF7B1FF09E0214628463F
:104A5000FFF7B0F904E021462846FFF7E2F900BF6E
:104A600000BF04E021462846FFF7DBF900BF00BF86
:104A7000304670BD2DE9F04105460E464FF0000866
:104A80003479307800F0600060B1202802D04028EE
:104A900071D100E000BFD5F8B402314682682846E3
:104AA000904700E1307800F06000202809D1D5F867
:104AB000B402314682682846904780464046BDE8A9
:104AC000F081707800285ED001282FD0032876D19D
:104AD00095F89C02022802D0032820D110E054B19E
:104AE000802C08D021462846FFF74AFE8021284620
:104AF000FFF746FE03E031462846FFF792F913E040
:104B0000708840B93CB1802C05D0F08818B9214696
:104B10002846FFF735FE2846FFF7C1F904E0314685
:104B20002846FFF77EF900BF00BFB5E095F89C026C
:104B3000022802D003281FD110E054B1802C08D0E5
:104B400021462846FFF71CFE80212846FFF718FE65
:104B500003E031462846FFF764F912E0708848B94F
:104B600004F07F0018B121462846FFF7E1FB2846F4
:104B7000FFF795F905E091E031462846FFF751F936
:104B800000BF00BF88E095F89C02022802D00328ED
:104B900076D126E034B1802C04D031462846FFF788
:104BA00040F972E004F08000802809D104F07F0011
:104BB00000EB800105F1140000EB810008E066E0E5
:104BC00004F07F0000EB800105F5AA7000EB810086
:104BD000074600203860022239462846FFF74EF982
:104BE00053E004F0800080280ED104F00F0000EBA9
:104BF000800105F1140000EB8100406898B931464E
:104C00002846FFF70EF940E004F00F0000EB8001AA
:104C100005F5AA7000EB8100406820B931462846AE
:104C2000FFF7FFF831E004F08000802808D104F09D
:104C30007F0000EB800105F1140000EB810007E02C
:104C400004F07F0000EB800105F5AA7000EB810005
:104C500007460CB1802C02D10020386009E02146C3
:104C60002846FFF7A9FC10B10120386001E00020C0
:104C70003860022239462846FFF700F905E0FFE7D1
:104C800031462846FFF7CDF800BF00BF04E03146AB
:104C90002846FFF7C6F800BF00BF04E031462846AB
:104CA000FFF7BFF800BF00BF404608E770B50546F4
:104CB0000C460026207800F0600030B1202802D099
:104CC00040282AD100E000BF00BF95F89C020128CF
:104CD00004D0022803D0032818D101E000BF00BF90
:104CE000207901280DDCD5F8B402214682682846D7
:104CF00090470646E08840B93EB92846FFF7CFF80E
:104D000003E021462846FFF78CF804E021462846B8
:104D1000FFF787F800BF00BF04E021462846FFF7F1
:104D200080F800BF00BF002070BD704701460148F9
:104D30007047000030140020F0B5024600260878C5
:104D4000400032F8100048F68F1400EA0403C878D7
:104D500030B101280CD0022805D003280BD104E083
:104D600043F4007309E000BF07E043F4C06304E0CC
:104D700043F4806301E0012600BF00BF43F400401C
:104D800040F080000C78640022F8140000BF0C781A
:104D9000640032F8144048F68F752C400D7844EAD0
:104DA000050040F4004444F080040D786D0022F8C2
:104DB000154000BF087B00287ED14878002852D0DB
:104DC00000BF1046B2F8505028440D7800F58067B7
:104DD00007EB0514CD886D106D00258000BF00BF66
:104DE0000C78640032F8140000F040048CB100BF6D
:104DF0000D786D0032F8155048F68F7705EA0704F4
:104E000044F4004545F0C0050F787F0022F81750A4
:104E100000BF00BFC878012813D000BF0C78640021
:104E200032F8144048F6BF7504EA050080F020000F
:104E300040F4004444F080040D786D0022F81540E1
:104E4000D0E100BF0C78640032F8144048F6BF751A
:104E500004EA050040F4004444F080040D786D003D
:104E600022F81540BEE100BF1046B2F85050284469
:104E70000D78042707EBC50500F5806707EB4504AF
:104E8000CD886D106D00258000BF00BF1546B2F8BB
:104E9000504025440C78062707EBC40405F58067CD
:104EA00007EB4404204600BF0788C7F309070780C3
:104EB0000F693E2F14D900E073E000BF0F697C0931
:104EC0000F7C07F01F0707B9641E07884FF4004CDA
:104ED0004CEA842C1FFA8CFC47EA0C07078017E089
:104EE0000F6927B9078847F40047078010E000BF23
:104EF0000F697C080F7C07F0010707B1641C078865
:104F00004FF6FF7C0CEA842C47EA0C07078000BFB1
:104F100000BF00BF00BF0C78640032F8140000F43A
:104F200080448CB100BF0D786D0032F8155048F602
:104F30008F7705EA070444F4004545F481450F786E
:104F40007F0022F8175000BF00BF0878A8B900BF43
:104F50000C78640032F814404BF68F7504EA0500B3
:104F600080F4805080F4005040F4004444F0800409
:104F70000D786D0022F8154034E100BF0C78640014
:104F800032F814404BF68F7504EA050080F40050A7
:104F900040F4004444F080040D786D0022F8154080
:104FA00020E1C878022811D100BF0C78640032F8E3
:104FB000144048F68F7504EA050040F4004444F4B8
:104FC000C0740D786D0022F8154011E000BF0C7818
:104FD000640032F8144048F68F6504EA050040F496
:104FE000004444F080040D786D0022F8154000BFA5
:104FF00000BF00BF00BF1046B2F8505028440D78E3
:1050000000F5806707EB05140D896D106D00258094
:1050100000BF00BF00BF00BF1046B2F85050284488
:105020000D78042707EBC50500F5806707EB4504FD
:105030004D896D106D00258000BF00BF00BF48780E
:10504000E8BB00BF0C78640032F8140000F4804420
:105050008CB100BF0D786D0032F8155048F68F778F
:1050600005EA070444F4004545F481450F787F00C4
:1050700022F8175000BF00BF00BF0C78640032F860
:10508000140000F040048CB100BF0D786D0032F8C0
:10509000155048F68F7705EA070444F4004545F0BB
:1050A000C0050F787F0022F8175000BF00BF00BF77
:1050B0000C78640032F814404BF68F7500E020E065
:1050C00004EA050080F4805080F4005040F400446D
:1050D00044F080040D786D0022F8154000BF00BF39
:1050E0000C78640032F8144048F6BF7504EA0500F5
:1050F00040F4004444F080040D786D0022F815401F
:1051000070E000BF0C78640032F8140000F48044B2
:105110008CB100BF0D786D0032F8155048F68F77CE
:1051200005EA070444F4004545F481450F787F0003
:1051300022F8175000BF00BF00BF0C78640032F89F
:10514000140000F040048CB100BF0D786D0032F8FF
:10515000155048F68F7705EA070444F4004545F0FA
:10516000C0050F787F0022F8175000BF00BFC87835
:10517000012813D000BF0C78640032F8144048F6C0
:10518000BF7504EA050080F0200040F4004444F0BC
:1051900080040D786D0022F8154011E000BF0C78F6
:1051A000640032F8144048F6BF7504EA050040F484
:1051B000004444F080040D786D0022F8154000BFD3
:1051C00000BF0C78640032F814404BF68F7504EA87
:1051D000050040F4004444F080040D786D0022F88E
:1051E000154000BF3046F0BD10B50446002010BD8C
:1051F00030B50246087B00285BD1487860B300BF19
:105200000B785B0032F8130000F040038BB100BF55
:105210000C78640032F8144048F68F7504EA0503F0
:1052200043F4004444F0C0040D786D0022F81540AA
:1052300000BF00BF00BF0B785B0032F8133048F6A8
:10524000BF7403EA040040F4004343F080030C7889
:10525000640022F8143007E100BF0B785B0032F8DD
:10526000130000F480438BB100BF0C78640032F867
:10527000144048F68F7504EA050343F4004444F4EF
:1052800081440D786D0022F8154000BF00BF00BFBB
:105290000B785B0032F813304BF68F7403EA04008E
:1052A00040F4004343F080030C78640022F814308B
:1052B000DAE0487800286BD100BF0B785B0032F849
:1052C000130000F480438BB100BF0C78640032F807
:1052D000144048F68F7504EA050343F4004444F48F
:1052E00081440D786D0022F8154000BF00BF00BF5B
:1052F0000B785B0032F8130000F040038BB100BF65
:105300000C78640032F8144048F68F7504EA0503FF
:1053100043F4004444F0C0040D786D0022F81540B9
:1053200000BF00BF00BF0B785B0032F8133048F6B7
:105330008F7403EA040040F4004343F0C0030C7888
:10534000640022F8143000BF00BF0B785B0032F815
:1053500013304BF68F7403EA040040F4004343F02B
:1053600080030C78640022F8143000BF00BF0B7873
:105370005B0032F8133048F6BF7403EA040040F4CF
:10538000004343F080030C78640022F814306BE093
:1053900000BF0B785B0032F8130000F480438BB140
:1053A00000BF0C78640032F8144048F68F7504EAA8
:1053B000050343F4004444F481440D786D0022F861
:1053C000154000BF00BF00BF0B785B0032F8130030
:1053D00000F040038BB100BF0C78640032F8144039
:1053E00048F68F7504EA050343F4004444F0C00412
:1053F0000D786D0022F8154000BF00BF00BF0B788C
:105400005B0032F8133048F68F7403EA040040F46E
:10541000004343F481430C78640022F8143000BF49
:1054200000BF0B785B0032F8133048F6BF7403EA14
:10543000040040F4004343F080030C78640022F839
:10544000143000BF00BF0B785B0032F813304BF60E
:105450008F7403EA040040F4004343F080030C78A7
:10546000640022F8143000BF002030BD0146002047
:10547000704701460020704710B50446012024F80B
:10548000400F00202080A0802082403C10BD0146BB
:105490004FF43F42B1F840009043A1F84000002093
:1054A000704702460020704730B50246087B00284E
:1054B00065D1487888B300BF0B785B0032F81300E1
:1054C00000F040038BB100BF0C78640032F8144048
:1054D00048F68F7504EA050343F4004444F0C00421
:1054E0000D786D0022F8154000BF00BFC878012874
:1054F00045D000BF0B785B0032F8133048F6BF741C
:1055000003EA040080F0200040F4004343F08003ED
:105510000C78640022F8143031E0FFE700BF0B780C
:105520005B0032F8130000F480438BB100BF0C78AD
:10553000640032F8144048F68F7504EA050343F41A
:10554000004444F481440D786D0022F8154000BFFA
:1055500000BF00BF0B785B0032F813304BF68F743E
:1055600003EA040080F4805080F4005040F40043CB
:1055700043F080030C78640022F8143000BF002050
:1055800030BD10B50246487898B100BF0B785B007B
:1055900032F8133048F6BF7403EA040080F01000BC
:1055A00040F4004343F080030C78640022F8143088
:1055B00013E000BF0B785B0032F813304BF68F74AA
:1055C00003EA040080F4805040F4004343F0800379
:1055D0000C78640022F8143000BF002010BD2DE9C3
:1055E000F04706460C466078012872D12169A0690F
:1055F000884201D9256900E0A569207BA0B9ABB23A
:10560000E2883046616900F056FD00BF3046B6F8CA
:10561000502010442278022303EBC20200F580637D
:1056200003EB42010D80C1E2E078022870D12169CC
:10563000206A88426DD900BF2178490036F81110E0
:1056400048F68F7201EA020040F4004141F4C07153
:105650002278520026F8121000BF206A401B2062F8
:105660002078400036F8100000F04000002874D088
:1056700000BF3346607868BB00BF3246B6F85010B2
:105680000A4421784FF0060909EBC10102F580694F
:1056900009EB4101084600BFB0F80090C9F30909C1
:1056A000A0F800903E2D16D900BF690905F01F092A
:1056B000B9F1000F00D1491EB0F800904FF4004A34
:1056C0004AEA812A1FFA8AFA49EA0A09A0F80090F0
:1056D0001CE081E21EE035B9B0F8009049F40049C1
:1056E000A0F8009012E000BF690805F00109B9F1C7
:1056F000000F00D0491CB0F800904FF6FF7A0AEA7C
:10570000812A49EA0A09A0F8009000BF00BF11E011
:105710007EE153E1607801280CD1B6F850000344D3
:105720002078062101EBC00003F5806101EB400CFD
:10573000ACF8005000BF6789ABB23A4630466169A9
:1057400000F0B9FC6069284460612169206A8842E0
:1057500004D9206A401B206203E05EE0256A002035
:10576000206200BF6078E0BB00BF3246B6F8501040
:105770000A442178022303EBC10102F5806303EBA5
:105780004101084600BF0388C3F3090303803E2D8F
:1057900010D900BF690905F01F0303B9491E03882A
:1057A0004FF4004C4CEA812C1FFA8CFC43EA0C03AA
:1057B000038014E025B9038843F4004303800EE01E
:1057C00000BF690805F0010303B1491C03884FF6C7
:1057D000FF7C0CEA812C43EA0C03038000BF00BF6E
:1057E00012E0FFE7607801280ED100BF3046B6F81E
:1057F000502010442278022303EBC20200F580639C
:1058000003EB42010D8000BF00BF2789ABB23A46CF
:105810003046616900F04FFCC8E100BF6078E0BB32
:1058200000BF3246B6F850100A442178022303EB39
:10583000C10102F5806303EB4101084600BF038804
:10584000C3F3090303803E2D10D900BF690905F099
:105850001F0303B9491E03884FF4004C4CEA812C06
:105860001FFA8CFC43EA0C03038014E025B903887B
:1058700043F4004303800EE000BF690805F0010314
:1058800003B1491C03884FF6FF7C0CEA812C43EAE4
:105890000C03038000BF00BF12E0FFE7607801281F
:1058A0000ED100BF3046B6F85020104422780223B3
:1058B00003EBC20200F5806303EB42010D8000BFE1
:1058C00000BF2789ABB23A463046616900F0F3FB6E
:1058D0006069284460612169206A884203D9206A8E
:1058E000401B206202E0256A0020206200BF334690
:1058F0006078A0BB00BF3246B6F850100A44217849
:105900004FF0060909EBC10102F5806909EB41017D
:10591000084600BFB0F80090C9F30909A0F800904C
:105920003E2D14D900BF690905F01F09B9F1000F18
:1059300000D1491EB0F800904FF4004A4AEA812A8B
:105940001FFA8AFA49EA0A09A0F800901BE03DB95B
:10595000B0F8009049F40049A0F8009013E014E07A
:1059600000BF690805F00109B9F1000F00D0491C1A
:10597000B0F800904FF6FF7A0AEA812A49EA0A094C
:10598000A0F8009000BF00BF0FE0607801280CD1A4
:10599000B6F8500003442078062101EBC00003F55F
:1059A000806101EB400CACF8005000BF6789ABB2DE
:1059B0003A463046616900F07EFBF7E0256A00BF99
:1059C0002178490036F8111048F68F6201EA02008A
:1059D00040F4004141F080012278520026F8121074
:1059E00000BF00BF3046B6F8502010442278022392
:1059F00003EBC20200F5806303EB42010D8000BFA0
:105A00002789ABB23A463046616900F054FBCDE0DD
:105A1000206A401B20622078400036F8100000F019
:105A2000400080B300BF3346607868BB00BF324699
:105A3000B6F850100A4421784FF0060909EBC1016D
:105A400002F5806909EB4101084600BFB0F80090FB
:105A5000C9F30909A0F800903E2D16D900BF6909C5
:105A600005F01F09B9F1000F00D1491EB0F80090F0
:105A70004FF4004A4AEA812A1FFA8AFA49EA0A09D7
:105A8000A0F800901CE036E01CE035B9B0F80090BA
:105A900049F40049A0F8009012E000BF690805F041
:105AA0000109B9F1000F00D0491CB0F800904FF681
:105AB000FF7A0AEA812A49EA0A09A0F8009000BFA1
:105AC00000BF0FE0607801280CD1B6F85000034405
:105AD0002078062101EBC00003F5806101EB400C4A
:105AE000ACF8005000BF6789ABB23A4630466169F6
:105AF00000F0E1FA5AE000BF6078E0BB00BF324638
:105B0000B6F850100A442178022303EBC10102F5D4
:105B1000806303EB4101084600BF0388C3F3090318
:105B200003803E2D10D900BF690905F01F0303B99A
:105B3000491E03884FF4004C4CEA812C1FFA8CFC60
:105B400043EA0C03038014E025B9038843F40043BF
:105B500003800EE000BF690805F0010303B1491C92
:105B600003884FF6FF7C0CEA812C43EA0C03038088
:105B700000BF00BF12E0FFE7607801280ED100BF30
:105B80003046B6F8502010442278022303EBC202BC
:105B900000F5806303EB42010D8000BF00BF278941
:105BA000ABB23A463046616900F085FA00BF217811
:105BB000490036F8111048F6BF7201EA020080F081
:105BC000100080F0200040F4004141F08001227874
:105BD000520026F8121028E2207B88BB2169A069B8
:105BE000884204D92569A069401BA06102E0A5692B
:105BF0000020A06100BF3246B6F850100A44217858
:105C0000062303EBC10102F5806303EB4101084663
:105C100000BF0388C3F3090303803E2D11D900BFE1
:105C2000690905F01F0303B9491E03884FF4004CAE
:105C30004CEA812C1FFA8CFC43EA0C03038015E02C
:105C400016E025B9038843F4004303800EE000BF4B
:105C5000690805F0010303B1491C03884FF6FF7C76
:105C60000CEA812C43EA0C03038000BF00BFC6E1AD
:105C7000E07802287CD100BF00BF607878BB00BF0D
:105C80003246B6F850100A442178022303EBC101D2
:105C900002F5806303EB4101084600BF0388C3F3AC
:105CA0000903038023693E2B12D900BF23695909D8
:105CB000237C03F01F0303B9491E03884FF4004CF3
:105CC0004CEA812C1FFA8CFC43EA0C03038018E099
:105CD00023692BB9038843F40043038011E012E0E9
:105CE00000BF23695908237C03F0010303B1491C59
:105CF00003884FF6FF7C0CEA812C43EA0C030380F7
:105D000000BF00BF12E0607801280FD100BF30460D
:105D1000B6F8502010442278022303EBC20200F5AB
:105D2000806303EB4201228A0A8000BF00BF00BFEC
:105D300033466078B0BB00BF3246B6F850100A4414
:105D400021784FF0060909EBC10102F5806909EBE2
:105D50004101084600BFB0F80090C9F30909A0F856
:105D60000090D4F81090B9F13E0F1CD900BF00E0AC
:105D70007BE0D4F810904FEA591194F8109009F094
:105D80001F09B9F1000F00D1491EB0F800904FF47F
:105D9000004A4AEA812A1FFA8AFA49EA0A09A0F85F
:105DA000009024E025E0D4F81090B9F1000F06D15E
:105DB000B0F8009049F40049A0F8009017E000BF47
:105DC000D4F810904FEA590194F8109009F00109A5
:105DD000B9F1000F00D0491CB0F800904FF6FF7ADF
:105DE0000AEA812A49EA0A09A0F8009000BF00BF28
:105DF00010E0607801280DD1B6F8500003442078F7
:105E0000062101EBC00003F5806101EB400C208A04
:105E1000ACF8000000BF00BFE069002824D0207863
:105E2000400036F8108008F4804010B108F04000BF
:105E300038B908F48040002816D108F04000002846
:105E400012D100BF00BF2178490036F8111048F682
:105E50008F7201EA020040F4004141F0C001227853
:105E6000520026F8121000BFC9E0E07801287ED168
:105E70002169A069884204D92569A069401BA061F5
:105E800002E0A5690020A06100BF00BF6078E0BB10
:105E900000BF3246B6F850100A442178022303EBC3
:105EA000C10102F5806303EB4101084600BF03888E
:105EB000C3F3090303803E2D10D900BF690905F023
:105EC0001F0303B9491E03884FF4004C4CEA812C90
:105ED0001FFA8CFC43EA0C03038014E025B9038805
:105EE00043F4004303800EE000BF690805F001039E
:105EF00003B1491C03884FF6FF7C0CEA812C43EA6E
:105F00000C03038000BF00BF12E0FFE760780128A8
:105F10000ED100BF3046B6F850201044227802233C
:105F200003EBC20200F5806303EB42010D8000BF6A
:105F300000BF00BF3346607870BB00BF3246B6F882
:105F400050100A4421784FF0060909EBC10102F50F
:105F5000806909EB4101084600BFB0F80090C9F321
:105F60000909A0F800903E2D17D900BF00E043E0DA
:105F7000690905F01F09B9F1000F00D1491EB0F8F9
:105F800000904FF4004A4AEA812A1FFA8AFA49EA45
:105F90000A09A0F800901BE01CE035B9B0F80090A9
:105FA00049F40049A0F8009012E000BF690805F02C
:105FB0000109B9F1000F00D0491CB0F800904FF66C
:105FC000FF7A0AEA812A49EA0A09A0F8009000BF8C
:105FD00000BF0FE0607801280CD1B6F850000344F0
:105FE0002078062101EBC00003F5806101EB400C35
:105FF000ACF8005000BF02E00120BDE8F08700BF10
:106000002178490036F811104BF68F7201EA020030
:1060100080F4805080F4005040F4004141F0800151
:106020002278520026F8121000BF0020E5E7014652
:106030000020A1F844004FF43F42A1F840207047EF
:1060400010B50248FBF7F5FB10BD00004011002021
:106050000146B1F8440070472DE9F04304460E466E
:1060600015464FEA530CA046304608F5806909EB07
:10607000450267460AE01188921C0170401C4FEAF5
:10608000112980F80090401C921C7F1E002FF2D135
:1060900003F00109B9F1000F01D011880170BDE8CA
:1060A000F083024600207047024611B98020A2F812
:1060B0004C00002070472DE9F04304460D461E4673
:1060C00006F101094FEA590CA046284608F58069F7
:1060D00009EB420367460AE0017890F8019041EA33
:1060E000092119809B1C9B1C401C401C7F1E002FFB
:1060F000F2D1BDE8F08300BFFEE70000024800686F
:10610000C0F30220704700000CED00E010B500283D
:1061100004DB0A07130E054A135406E00A07140E9F
:10612000034A00F00F031B1FD45410BD00E400E02D
:1061300018ED00E002E008C8121F08C1002AFAD1D9
:1061400070477047002001E001C1121F002AFBD1F7
:106150007047014609B90120704700200860486077
:1061600000BFF9E703460BB101B10AB9012070473E
:10617000501E104008B10220F9E79A60D960002053
:106180001860586000BFF2E7024602B109B9012069
:106190007047D2E90003C01A08600020F8E72DE933
:1061A000F04103469446D3E90008A0EB0800904272
:1061B00001D9104603E0D3E90008A0EB080002462D
:1061C000D3E90108A8F1010800EA0800D3F8088023
:1061D000A8EB0000904201D9104609E0D3E901087C
:1061E000A8F1010800EA0800D3F80880A8EB000035
:1061F0000746D3E90108A8F1010800EA0800D3F82E
:106200000C8000EB0805002404E015F8010B01F8F0
:10621000010B641CBC42F8D3D61B4EB1DD680024D0
:1062200004E015F8010B01F8010B641CB442F8D32B
:10623000586810445860624502D20420BDE8F081DD
:106240000020FBE72DE9F04103469446D3F8008097
:106250009868A0EB0800D3F804804044904201D92C
:10626000104607E0D3F800809868A0EB0800D3F848
:10627000048040440246D3F80880A8F10108186859
:1062800000EA0800D3F80880A8EB0000904201D98A
:1062900010460AE0D3F80880A8F10108186800EA5F
:1062A0000800D3F80880A8EB00000746D3F8088060
:1062B000A8F10108186800EA0800D3F80C8000EB88
:1062C0000805002404E011F8010B05F8010B641C1B
:1062D000BC42F8D3D61B4EB1DD68002404E011F8AF
:1062E000010B05F8010B641CB442F8D31868104484
:1062F0001860624502D20320BDE8F0810020FBE770
:1063000010B5012240210248FAF7E2FC10BD00005E
:10631000000C014010B5002240210248FAF7D8FCD9
:1063200010BD0000000C014010B5012220210248E0
:10633000FAF7CEFC10BD0000000C0140144951F8E2
:106340003010491C124A42F83010114651F83010F2
:1063500064291BD9114601EBC001097969B91146BD
:1063600001EBC001897989B9012102EBC002917169
:10637000074A02EBC002517108E00121044A02EB16
:10638000C00251710021024A42F8301070470000EB
:10639000AC0100200021034A42F8301002EBC00299
:1063A00091717047AC01002010B510211248FAF726
:1063B00087FC18B90020FFF7C1FF02E00020FFF7BB
:1063C000E9FF4FF400710C48FAF77AFC18B9012084
:1063D000FFF7B4FF02E00120FFF7DCFF8021064851
:1063E000FAF76EFC18B90220FFF7A8FF02E00220BE
:1063F000FFF7D0FF10BD0000000C0140FAF780FC51
:10640000FCF7E3FFFCF742FCFCF700FDFCF71AFD8C
:10641000FCF7BEFC002000F04BF9012207490848B8
:10642000FCF796FB002000F073F900F0C1F904E0DE
:1064300000F0CEF90120FAF79FFAF9E704000020F6
:106440000C0200200748006850B106480068401E52
:10645000044908600846006810B901200249087024
:1064600070470000A4010020A801002010B50221FF
:106470000D48FAF725FCA0B9FAF730FC044607E00E
:10648000FAF72CFC001B642802D36FF0010010BD4A
:1064900002210548FAF714FC0028F1D00220FAF78F
:1064A0006BFA0020F3E70000000C0140054800787B
:1064B00010B94FF0FF30704700200249087000BF4C
:1064C000F9E70000A001002010B50548FFF741FEE4
:1064D000044614B14FF0FF3010BD0020FCE700006F
:1064E000501E002038B5044614B96FF0020038BDC4
:1064F00069460648FFF748FE054615B14FF0FF30E4
:10650000F5E7009820800020F1E70000501E0020F1
:10651000F8B507460D4614460FB105B114B96FF032
:106520000200F8BD69461048FFF72EFE064616B178
:106530004FF0FF30F5E7009818B900202080401E8A
:10654000EFE70098A84200D9009539460648009A1E
:10655000FFF725FE06461EB100202080401EE0E722
:10656000009820800020DCE7501E002010B50B486A
:10657000007810B14FF0FF3010BD4FF48062084931
:106580000848FFF7EFFD044614B14FF0FF30F3E782
:106590000120024908700020EEE70000A001002061
:1065A000501A0020501E002070B50546FFF75EFF10
:1065B00004460CB1204670BD35B1012D0FD0022D1F
:1065C00018D0032D2CD120E0002280211C48FAF79E
:1065D0007FFB002201211B48FAF77AFB23E001220E
:1065E00080211748FAF774FB002201211548FAF7B9
:1065F0006FFB18E0002280211148FAF769FB0122A5
:1066000011461048FAF764FB0DE0012280210C4886
:10661000FAF75EFB012211460A48FAF759FB02E03D
:106620006FF00200C7E700BF0520FAF7A5F9FFF7F2
:106630001DFF04460CB12046BDE70020BBE700006B
:1066400000080140000C014008B509480068406896
:10665000C0B20090012269460648FFF7F3FD0A2008
:1066600005490860012205490148FCF771FA08BD97
:106670000C020020501E0020A4010020A1010020D7
:1066800070B504460D4604B115B96FF0020070BD37
:106690004FF6FF732A4621460448FCF77BFA06466C
:1066A00016B16FF00100F2E70020F0E70C020020C5
:1066B00070B505461348007810B14FF0FF3070BD3B
:1066C000FFF754FF044614B14FF0FF30F7E735B938
:1066D0000D480E490A6802600979017104E00A4810
:1066E0002968016029790171074800F0F1F8044632
:1066F0001CB1FFF7DBFE2046E1E7012001490870ED
:106700000020DCE790010020910100202E6A0008A3
:1067100070B5054615B94FF0FF3070BD28210F4800
:10672000F9F71BFD00200D49087081F82500084687
:1067300029680162297980F82410203000F0C8F817
:1067400004460CB12046E8E7002000F0EDF80446CE
:106750000CB12046E1E70020DFE7000054020020F2
:106760002DE9F04104460D4616461F4614B10DB101
:1067700006B11FB94FF0FF30BDE8F0810A2D02DAF3
:106780004FF0FF30F8E72078542802D1607858287D
:1067900002D04FF0FF30EFE73B46324602A1E01C4B
:1067A000F9F7E6FC0020E7E725642E25642E0000BB
:1067B00010B500F05DF804460CB1204610BD012074
:1067C0000249087081F825000020F7E754020020F4
:1067D00010B594B0254890F8250008B914B010BD44
:1067E0002248007820B1012806D0022836D134E0B2
:1067F00001201E49087035E00020039003A904A879
:1068000000F0D4F840B3002002900190039881B2C8
:1068100001AB02AA04A8FFF7A3FF0446DCB91348A2
:106820004068401C1149486002988861019848619D
:106830000846C0690199884202D20C490198C86192
:1068400000F088F8012000F07BF83220FAF794F885
:10685000002000F075F800BF04E003E002200349C7
:10686000087000BF00BF00BFB8E70000540200205E
:1068700010B50C48007810B96FF0050010BD0A483B
:10688000007810B16FF00100F8E7FFF71DFE044635
:1068900014B14FF0FF30F1E70120034908700020E8
:1068A000ECE70000900100209601002010B504469E
:1068B000C0200649087008462168C0F801102179F7
:1068C00041710621FFF7DCFE10BD000050160020CC
:1068D00070B5054615B96FF0030070BDFFF7C6FD32
:1068E000044614B16FF00200F7E70320FFF75CFEE7
:1068F000044614B16FF00200EFE72846FFF7D6FF19
:106900006420FAF739F80020FFF74EFE044614B170
:106910006FF00200E1E703482968016029790171FD
:106920000020DAE79101002070B504462046FFF709
:106930003BFE054615B16FF0020070BD0020FCE77C
:1069400010B5044614B1FFF7E5FC01E0FFF7D8FCF1
:1069500010BD00000D48C069B8B10C48C0690B49B2
:106960004968411A0948C160C06958B10748C06800
:10697000642148430549C969B0FBF1F0C1B203483D
:10698000017402E0002101480174704754020020A4
:1069900010B500F033F80448006820B102480068E0
:1069A000401E0149086010BD00000020F8B50646F1
:1069B0000D4606B10DB90020F8BD0F48007808B9A2
:1069C0000020F9E76846FFF78DFD04460CB1002072
:1069D000F2E7BDF8000008B90020EDE72A46FF21E4
:1069E0003046FFF795FD04460CB10020E4E7002097
:1069F000014908700120DFE7A801002000B5FFF77A
:106A000021FD00BD02030405060708090A0B0C0D51
:106A10000E0F101001020000000000000000010233
:106A20000304060708090000000001020304000037
:106A30001A1704C1C1C141542B44455654595045FD
:106A40003D3F0041542B4657434F44453D3F00DDF9
:106A5000DDDDDDDCBBBBDDDDDDDDDDDDDDDDDD98F0
:106A600088888888888888777777777788888885FE
:106A70005555566666666666666666666888888385
:106A800033333222222222222222222228888D00FF
:106A9000B06A000800000020AC01000000070008F8
:106AA000746B0008AC010020B420000044610008B1
:106AB00051220113ED3E1408353F1B0845041A719D
:106AC000041AB1041AB9141AFD04131201140202B3
:106AD000021640830440571D0201020330071E04C2
:106AE0000309041A0313A5071B089F041A5B041A61
:106AF000C904414A106F215324F4130A0632022AB2
:106B000040141B893B28123A4C08AB3C2C1A171036
:106B10001A19101A9504C11A69181A59041A790415
:106B20001A49041C09024397111DC03209045D1A59
:106B3000020B130524161001052401100901042479
:106B40000202052406170107058203081C10090428
:106B5000CD320A1D070501027B2C070581071109AB
:106B600037442A40072A8107112B0907440A3B04AE
:046B700044011C00C0
:04000005080000ED02
:00000001FF
